:100000000C94D0010C9414020C9414020C9414025D
:100010000C9414020C9414020C9414020C94140208
:100020000C9414020C9414020C94950C0C94670D0F
:100030000C9414020C9414020C9414020C941402E8
:100040000C9414020C9421210C9414020C941402AC
:100050000C9414020C94B41A0C9414020C94140210
:100060000C9414020C9414020C9414020C941402B8
:100070000C9414020C9414020C9414020C941402A8
:100080000C9414020C9414020C9414020C94140298
:100090000C9414020C9414020C9414020C94140288
:1000A0000C9414020C9414020C941402D40DF60D4A
:1000B000E40EF60DE40E3B0E5E0EE40EB30EC60E1D
:1000C00095119511C411C411FA111A124B134B1347
:1000D00025124B13D512D5123C134B134B1345135A
:1000E000E212E212E212E212E212E212E212E21270
:1000F000E212E212E212E212E212E212E212E21260
:10010000F412011308130F13191335002B00297172
:10011000E1003A0000001E00140004001D003B0036
:10012000E2001F001A0016001B003C00297120008D
:100130000700080006003D002A0021000900170002
:100140001900E300A90022000E000A0005000000CB
:10015000AA003E00310000002F000000A8003F0070
:100160000000000030000000AE0023000D001C0065
:1001700013000000AB002400180011001000E7007D
:10018000AC00250015000C00360050002C002600A5
:100190000F001200370051003400270033000B001D
:1001A00038005200E6002E002D002800E5004F0028
:1001B000000016034500720067006F0044006F00E6
:1001C0007800200045005A00000016034500720028
:1001D00067006F0044006F007800200045005A005F
:1001E00000000403090409026D00040100A0FA09DB
:1001F0000400000103010100092111010001223F57
:10020000000705810308000A090401000103010237
:1002100000092111010001224D0007058203080099
:100220000A09040200010300000009211101000174
:100230002236000705830308000A090403000103AE
:100240000000000921110100012239000705840383
:100250001000011201100100000008EDFE0713015B
:10026000000102000105010906A101050719E029A5
:10027000E715002501950875018102050819012976
:100280000595057501910295017503910105071901
:1002900000297715002501957875018102C00501B7
:1002A0000980A101850216010026B7001A01002A63
:1002B000B700751095018100C0050C0901A10185E9
:1002C00003160100269C021A01002A9C0275109553
:1002D000018100C005010902A1010901A100050970
:1002E0001901290515002501950575018102950162
:1002F000750381010501093009311581257F9502BA
:100300007508810609381581257F950175088106D4
:10031000050C0A38021581257F950175088106C0F4
:10032000C005010906A101050719E029E715002507
:10033000019508750181029501750881010508196B
:100340000129059505750191029501750391010536
:1003500007190029FF150025FF950675088100C0C3
:100360000000000000000000000000010204060A76
:100370000F17202C3A4A5D71879DB3C7DAE9F5FC67
:10038000FFFCF5E9DAC7B39D87715D4A3A2C201767
:100390000F0A060402010000000000000000000037
:1003A00011241FBECFEFDAE0DEBFCDBF04B603FEDF
:1003B00024C08091FB019091FC01A091FD01B091BE
:1003C000FE018730904BA740B04BB9F41092FB016F
:1003D0001092FC011092FD011092FE0114BE84B730
:1003E000877F84BF88E10FB6F894809360001092F5
:1003F00060000FBEE0E0FFE3099511E0A0E0B1E08E
:10040000E0EDF5E402C005900D92A433B107D9F7F1
:1004100011E0A4E3B1E001C01D92AB3FB107E1F7E9
:100420000E94D9090C94E6220C9400001092B900A5
:100430008AE08093B800089594EA9093BC0090916C
:10044000BC0097FFFCCF9091B900987F983021F0C5
:10045000903111F081E008958093BB0084E880938F
:10046000BC008091BC0087FFFCCF8091B900887FE1
:10047000883111F0803471F780E0089584E9809329
:10048000BC008091BC0084FDFCCF08958093BB002C
:1004900084E88093BC008091BC0087FFFCCF9091E2
:1004A000B900987F81E0983209F480E0089584E8EB
:1004B0008093BC008091BC0087FFFCCF8091BB0083
:1004C000089580910101811115C080E40E941C02F1
:1004D0008093010181110CC082E10E944602809349
:1004E0000101811105C08FEF0E9446028093010136
:1004F0000E943E0284B1807F84B985B1807F85B936
:100500008AB1837F8AB98BB1837F8BB93E98469835
:1005100008950E941C04809301010E94610280B32F
:100520008C7080BB81B3836F81BBA5E3B1E0E3E452
:10053000F1E08EE08E0F11921D928E13FCCF0C9481
:100540000604BF92CF92DF92EF92FF920F931F9318
:10055000CF93DF9380910101882379F0809134015A
:100560008F5F80933401811108C00E941C04809326
:100570000101811102C00E94AE0305E311E0C0E059
:10058000D0E0DD24D39482E0C82EEE24E394F12C55
:10059000C730D10500F580910101811164C080E46C
:1005A0000E941C0280930101811112C082E10E940D
:1005B00046028093010181110BC0C7010C2E01C0BE
:1005C000880F0A94EAF780950E9446028093010101
:1005D0000E943E0248C0CA30A1F028F4C83059F049
:1005E000C93061F005C0CC3089F070F0CD3089F0B1
:1005F000209A289810C0219A29980DC0229A2A98EA
:100600000AC0239A2B9807C0529A01C0539A5B984C
:1006100002C03E9A469890EA9A95F1F79FB179996F
:1006200002C082E001C080E091709D25982B7C99EA
:1006300002C084E001C080E0892B7D9902C038E0CF
:1006400001C030E0832B7E9902C020E101C020E090
:10065000822B9FB19095991F9927991F9295990F79
:10066000907E892B0FC080910101811149C080E4E7
:100670000E941C0280930101882379F1B12C0E9411
:100680003E028B2DF8019081981719F08083C0925B
:1006900000010E94610221960F5F1F4FCE30D105ED
:1006A00009F076CF80910001882361F18150809319
:1006B0000001882339F08FE99FE00197F1F700C02E
:1006C000000020C0A3E4B1E0E5E3F1E0CF01825FE8
:1006D00091919D938E13FCCF15C083E10E94460239
:1006E000809301018111CACF81E40E941C02809392
:1006F00001018111C3CF0E945702B82EB094BFCF21
:1007000080E0C0CF0E94AC0381E0DF91CF911F91C8
:100710000F91FF90EF90DF90CF90BF900895E82F5A
:10072000F0E0ED5BFE4F8081089508950F931F93D5
:10073000CF93DF93C3E4D1E010E00C2F025F8991E7
:1007400090E00E942A1A180F0C13F9CF812FDF9125
:10075000CF911F910F9108950C94750456985E984F
:1007600025982D9826982E9827982F988FEF90E00F
:10077000909389008093880090938B0080938A00E7
:1007800090938D0080938C00259A2D9A2FEF80E70F
:1007900092E0215080409040E1F700C00000269A8E
:1007A0002E9A2FEF80E792E0215080409040E1F7B1
:1007B00000C00000279A2F9A2FEF80E792E0215087
:1007C00080409040E1F700C0000025982D982FEF61
:1007D00080E792E0215080409040E1F700C00000A7
:1007E00026982E982FEF80E792E02150804090408D
:1007F000E1F700C0000027982F9856985E9825983A
:100800002D9826982E9827982F98089589EA8093F6
:10081000800089E08093810024982C983F988AB1C9
:100820008F748AB96E98479A8BB1806B8BB9769A20
:100830000E94AE030C946C0480E2809301018091CD
:10084000510181110EC00E94160281E08093510176
:100850002FEF83ED90E3215080409040E1F700C0FE
:10086000000080E40E941C028093010181112EC0CF
:100870000E94460280930101811128C00E94460215
:1008800080930101811122C08FE30E944602809370
:10089000010181111BC00E943E0280E40E941C02E3
:1008A00080930101811112C08CE00E944602809366
:1008B000010181110BC00E94460280930101811148
:1008C00005C08FE30E944602809301010E943E0210
:1008D000809101010895089556985E9825982D9865
:1008E00026982E9827982F980895089581E00895C6
:1008F00081E008950C94780408950F931F93CF938B
:10090000DF938C01FC01C081D181CE010E94AF1820
:10091000BE010E942605EC01B8010E947A048823DA
:1009200009F48DC0F8018281882309F44AC08091BE
:100930005D0181111FC0C431F0E5DF0709F051C02E
:100940000E947C0481E080935D010E947E1A909356
:100950005C0180935B011092540110925601109239
:100960005501109258011092570110925A0110929D
:10097000590165C080915B0190915C010E948A1AC7
:10098000883C910570F480915401E82FF0E0EE0F5F
:10099000FF1FEB5AFE4FD183C0838F5F80935401BA
:1009A0004EC0C43880E5D80721F0C538D04501F1E4
:1009B0003AC0F8018281882341F01092520182E00E
:1009C0001EC0C438E0E5DE0759F58091520181115F
:1009D00006C086E20E94391086E20E94011182E080
:1009E0001CC0C438F0E5DF0741F3C538D045D9F461
:1009F000F8018281882331F01092530180E20E9435
:100A000050111DC080915301811106C087E20E94E0
:100A1000391087E20E94011180E20E9457110FC035
:100A2000C538D04529F381E080935201809353016A
:100A3000C801DF91CF911F910F910C94760480E053
:100A4000DF91CF911F910F910895089596E0799FBE
:100A5000F001112494E5899FE00DF11D1124E60FAA
:100A6000F11DEE0FFF1FE65FFE4F859194910895F3
:100A7000880F991FFC01E657F040859194910895E5
:100A8000880F991FFC01E65FFE4F859194910895B0
:100A90000F931F93CF93DF93EC01811520E392070F
:100AA00050F5C11580E2D80708F0C3C0CB3BD10593
:100AB00090F4C83AD10508F06AC0C53AD10508F0EB
:100AC0005BC0C430D10508F0D0C1219709F0CAC17C
:100AD00001E010E00AC2CF3FD10511F008F0C5C116
:100AE000C03FD10508F0A2C0CE01805E91090897F1
:100AF00008F4BBC1B7C1C13090E5D90709F4A2C061
:100B000020F5C0318FE4D80770F4C11590E4D907FF
:100B100008F094C0C11521E3D20708F0A3C1DD2776
:100B20008E01106CE2C1C115D04509F09BC10E9435
:100B3000B6138FEF94E32CE0815090402040E1F712
:100B400000C000000E94D91AD0C1C11597E5D9078D
:100B500058F4C03121E5D20708F01CC1C43180E54A
:100B6000D80708F475C07EC1CE0190578115904119
:100B700008F078C1DF7073C1C53AD10509F477C1B7
:100B8000C63AD10509F076C102E810E4AEC1C83A10
:100B9000D10509F472C1C93AD10509F471C1CA3A43
:100BA000D10509F470C1CB3AD10509F46FC1CC3A33
:100BB000D10509F46EC1CD3AD10509F46DC1C03B30
:100BC000D10509F46CC1CE3AD10509F46BC1CF3A15
:100BD000D10509F46AC1C13BD10509F469C1C23B21
:100BE000D10509F468C1C33BD10509F467C1C43B11
:100BF000D10509F466C1C53BD10509F465C1C63B01
:100C0000D10509F464C1C73BD10509F463C1C83BF0
:100C1000D10509F462C1C93BD10509F461C1CA3BE0
:100C2000D10509F460C100E014E45FC18E011065D4
:100C30005CC1CE019F700E94400558C1DF708E01DB
:100C4000106A53C18091DA0181608093DA014DC14D
:100C50000E947E1C811102C00E94641C0E949B1C89
:100C600090E09093FB018093FA01C23080E5D807B1
:100C700021F48091FA01816086C0C43090E5D907E3
:100C800021F48091FA0182607EC0C63020E5D2074F
:100C900021F48091FA01846076C0C83080E5D807DD
:100CA00019F48091FA0127C0CA3090E5D90721F4E0
:100CB0008091FA01806167C0CC3020E5D20721F431
:100CC0008091FA0180625FC0CE3080E5D80721F4C0
:100CD0008091FA01806457C0C03190E5D90721F4B2
:100CE0008091FA0180684FC0C23120E5D20729F413
:100CF0008091FA018460886046C0C33080E5D807DF
:100D000021F48091FA018E7F3EC0C53090E5D9076D
:100D100021F48091FA018D7F36C0C73020E5D207DB
:100D200021F48091FA018B7F2EC0C93080E5D8076D
:100D300019F48091FA0126C0CB3090E5D90721F44F
:100D40008091FA018F7E1FC0CD3020E5D20721F4BB
:100D50008091FA018F7D17C0CF3080E5D80721F44C
:100D60008091FA018F7B0FC0C13190E5D90721F442
:100D70008091FA018F7707C0C331D04531F480915B
:100D8000FA018B7F877F8093FA018091FA010E949C
:100D90009F1CABC08D2F99278F70992781309105AB
:100DA000D9F49E012370332702C0880F991F2A951A
:100DB000E2F79C688E0144E0000F111F4A95E1F7AD
:100DC00000271370802B912B53E0CC0FDD1F5A9519
:100DD000E1F7C076DD272FC08230910531F4DC2F9A
:100DE000CC278E01016F106A80C08330910569F4B1
:100DF000CE018370992701E010E002C0000F111F9F
:100E00008A95E2F7C8019C680FC084309105B9F457
:100E1000CE018370992701E010E002C0000F111F7E
:100E20008A95E2F7C8019A6823E0CC0FDD1F2A9566
:100E3000E1F7C07ED7708C010C2B1D2B56C085307E
:100E4000910531F4DC2FCC278E01046F106A4DC060
:100E5000069709F04AC0CF71DD27DC2FCC278E0121
:100E6000106243C000E010E040C08E013EC001E8C7
:100E700010E43BC003E810E438C002EE14E435C0CF
:100E800009EE14E432C00AEE14E42FC005EB14E4BA
:100E90002CC006EB14E429C007EB14E426C00CECCC
:100EA00014E423C00DEC14E420C003E815E41DC0D5
:100EB0000AE815E41AC002E915E417C004E915E4CC
:100EC00014C001E216E411C003E216E40EC004E20D
:100ED00016E40BC005E216E408C006E216E405C0FD
:100EE00007E216E402C00AE216E4C801DF91CF91DE
:100EF0001F910F91089596E0799FF001112494E5D8
:100F0000899FE00DF11D1124E60FF11DEE0FFF1F6B
:100F1000E65FFE4F85919491803E9105E0F4803C20
:100F2000910558F58133910509F46FC048F4893271
:100F3000910509F463C08A32910509F46DC072C04D
:100F400089339105E9F082389105D1F08533910517
:100F500009F44DC067C0833E910581F138F4803EAD
:100F60009105B9F0823E9105D9F05CC0863E9105AD
:100F700061F1873E9105A1F155C00E9438050895A1
:100F80002091FA0120FD02C021FF4CC080EE90E0CC
:100F900049C08091FA0180FFF9CF89E390E042C017
:100FA0008091FA0182FF0EC08091FA0184FF03C094
:100FB00080E090E037C083EE90E034C08091FA0189
:100FC00082FFF2CF82EE90E02DC08091FA0183FF84
:100FD0000BC08091FA0184FDEBCF87EE90E022C038
:100FE0008091FA0183FFF5CF86EE90E01BC08091DF
:100FF000FA0185FF07C089E290E014C08091FA01F0
:1010000085FFF9CF85E390E00DC08091FA0186FF5E
:1010100007C08AE290E006C08091FA0186FFF9CF0E
:1010200081E390E00E944805089508950C94150806
:1010300080916E010895CF93DF9300D01F92CDB7BA
:10104000DEB79C018091F101843019F593E099831A
:101050003B832A839093E9008FEF9091E8008150C1
:1010600095FD06C095ED9A95F1F700008111F5CF39
:101070008091E80085FF0DC040E050E063E070E043
:10108000CE0101960E94850A8091E8008E778093B8
:10109000E8000F900F900F90DF91CF910895CF93BC
:1010A000DF9300D01F92CDB7DEB72091F10124303D
:1010B00021F522E029839B838A8383E08093E900E2
:1010C0008FEF9091E800815095FD06C095ED9A95BF
:1010D000F1F700008111F5CF8091E80085FF0DC088
:1010E00040E050E063E070E0CE0101960E94850A86
:1010F0008091E8008E778093E8000F900F900F901A
:10110000DF91CF9108952091F1012430F1F422E094
:101110002093E9002FEF3091E800215035FD06C003
:1011200035ED3A95F1F700002111F5CF2091E80057
:1011300025FF0BC040E050E065E070E00E94850AAA
:101140008091E8008E778093E8000895CF93DF9335
:10115000EC019091F101943009F046C080910C01AE
:101160008823D9F080910D018823B9F09093E9008C
:101170008FEF9091E800815095FD06C095E19A951A
:10118000F1F700008111F5CF8091E80085FF2CC0B8
:1011900040E050E060E170E017C081E08093E9003A
:1011A0008FEF9091E800815095FD06C095ED9A95DE
:1011B000F1F700008111F5CF8091E80085FF14C0A0
:1011C00040E050E068E070E0CE010E94850A809126
:1011D000E8008E778093E80080E1FE01AEE5B1E0A3
:1011E00001900D928A95E1F7DF91CF91089580915A
:1011F000F001811109C00E941A0C0E94770C8091A5
:10120000E20084608093E20008951092F001089556
:1012100008950C940E210E946F1A0E9414210E94BE
:101220001D0F0C94160842E061EC81E00E94940BC3
:1012300042E061EC82E00E94940B42E061EC83E0CA
:101240000E94940B42E161EC84E00C94940B809139
:10125000F301833009F455C030F4813071F08230ED
:1012600009F48EC008958A3009F47AC08B3009F4ED
:1012700060C0893009F09CC020C08091F201813AA1
:1012800009F096C08091E800877F8093E800809104
:10129000F6019091F701892B21F460E18EE591E050
:1012A00003C060E080E090E070E00E94D00A80918E
:1012B000E8008B778093E80008958091F2018132F5
:1012C00009F076C08091F6019091F701009719F02E
:1012D000039709F06DC08091E800877F8093E80054
:1012E0008091E80082FD05C08091F1018111F8CF65
:1012F0005FC08091F10080936E018091E8008B7750
:1013000053C08091F201813A09F052C08091F601F8
:101310009091F701892B09F04BC08091E800877FFD
:101320008093E8008091E80080FFFCCF80910C0161
:1013300036C08091F2018132D9F58091F601909109
:10134000F701892BA9F58091E800877F8093E80059
:101350000E94C90B8091F40180930C010C94B61388
:101360008091F201813221F58091E800877F80939E
:10137000E8000E94C90B8091F50180936F010895E8
:101380008091F201813AA1F48091E800877F8093F7
:10139000E8008091E80080FFFCCF80916F0180938E
:1013A000F1008091E8008E778093E8000C94C90BDF
:1013B000089584B7877F84BF88E10FB6F89480933F
:1013C0006000109260000FBE90E080E80FB6F894C5
:1013D00080936100909361000FBE0E946C0F0E9489
:1013E0001A0C0E94770C8091E20084608093E200E6
:1013F00078940E94FD0E0E946E0F82E091E00E94A0
:10140000180F0E94FC208091F101853069F40E9440
:10141000361A8091EF018823B1F30E94611A882364
:1014200091F30E946F0AEFCF0E94740FECCF292F27
:10143000332723303105C9F064F42130310581F0C0
:101440002230310509F043C08DE690E026EE31E010
:1014500042C021323105F1F02232310541F137C06D
:1014600082E190E023E532E036C099278130910592
:1014700041F08230910541F0892B49F5E2EEF1E02F
:1014800005C0EAECF1E002C0E2EBF1E0849190E00B
:101490009F0121C06430D8F4E62FF0E0EE0FFF1F6B
:1014A000EE5DFE4F2081318189E090E014C0643010
:1014B00070F470E0FB01EE0FFF1FE65EFE4F20812F
:1014C0003181FB01EA5EFE4F808190E004C080E044
:1014D00090E020E030E0FA0131832083089580E13C
:1014E00089BD82E189BD09B400FEFDCF8091D8009D
:1014F0008F7D8093D8008091E00082608093E0002F
:101500008091E00081FDFCCF0895CF92DF92EF92B1
:10151000FF920F931F93CF93DF93EC018B016A012E
:101520000E94E80B811133C0C114D10439F0F601D7
:1015300080819181081B190BC80FD91FE12CF12C58
:101540000115110519F18091E80085FD16C0809103
:10155000E8008E778093E800C114D10449F0F601C9
:1015600080819181E80EF91EF182E08285E00FC052
:101570000E94E80B882321F30AC089918093F1002F
:1015800001501109FFEFEF1AFF0ADACF80E0DF9177
:10159000CF911F910F91FF90EF90DF90CF90089522
:1015A0002091F8013091F9012617370748F06115AD
:1015B000710539F42091E8002E772093E80001C0EE
:1015C000B90140E061157105A9F12091F1012223D3
:1015D00009F443C0253009F442C02091E80023FDFE
:1015E00040C02091E80022FD32C02091E80020FF99
:1015F000E9CF4091F3002091F20030E0342BFC0160
:10160000CF016115710559F02830310540F4819101
:101610008093F100615071092F5F3F4FF1CF41E09E
:101620002830310509F040E02091E8002E77209322
:10163000E800C8CF4111C9CF0AC08091F1018823C9
:1016400061F0853061F08091E80083FD0AC08091EF
:10165000E80082FFF2CF80E0089582E0089583E001
:10166000089581E008952091F8013091F90126173D
:10167000370748F06115710539F42091E8002E779D
:101680002093E80001C0B901FC0120E0611571055B
:1016900091F18091F101882309F440C0853009F46B
:1016A0003FC08091E80083FD3DC08091E80082FD4D
:1016B0002FC08091E80080FFE9CF2091F300809156
:1016C000F20090E0922B6115710559F08830910578
:1016D00040F424912093F1003196615071090196F4
:1016E000F2CF21E0089709F020E08091E8008E77A2
:1016F0008093E800CBCF2111CCCF0AC08091F101BB
:10170000882361F0853061F08091E80083FD0AC094
:101710008091E80082FFF2CF80E0089582E0089592
:1017200083E0089581E00895982F973058F59093BD
:10173000E900981739F07091EC002091ED0050917C
:10174000F00003C0242F762F50E021FF19C0309104
:10175000EB003E7F3093EB003091ED003D7F309306
:10176000ED003091EB0031603093EB007093EC00B2
:101770002093ED005093F0002091EE0027FF07C06A
:101780009F5FD3CF8F708093E90081E0089580E060
:1017900008958091F20187FF11C08091E80082FDD9
:1017A00005C08091F1018111F8CF11C08091E8004E
:1017B0008B770BC08091F101882349F08091E8007C
:1017C00080FFF8CF8091E8008E778093E80008953D
:1017D0002091E4003091E50095E64091EC00842FE3
:1017E000817040FF22C08091E80080FD1CC0809184
:1017F000F101882391F0853091F08091EB0085FD17
:1018000010C04091E4005091E5004217530729F3BE
:101810009A01915011F784E0089582E0089583E0E1
:10182000089581E0089580E008954091E80042FF26
:10183000DECF08950E94880C0E94900CE0EEF0E04C
:10184000808181608083E8EDF0E080818F77808304
:1018500019BCA7EDB0E08C918E7F8C9380818F7E38
:1018600080831092F00108950F931F93CF93DF931D
:101870000E94880C0E94900CC8EDD0E088818F7780
:10188000888388818068888388818F7D888319BC5C
:101890001092F1011092ED011092EF011092EE0101
:1018A00000EE10E0F80180818B7F80838881816069
:1018B000888342E060E080E00E94940BE1EEF0E07B
:1018C00080818E7F8083E2EEF0E080818160808382
:1018D000808188608083F80180818E7F8083888109
:1018E00080618883DF91CF911F910F910895E8ED7A
:1018F000F0E080818F7E8083E7EDF0E08081816081
:10190000808384E082BF81E08093F0010C94340CEA
:10191000E8EDF0E080818E7F80831092E2000895F0
:101920001092DA001092E10008951F920F920FB604
:101930000F9211242F933F934F935F936F937F9355
:101940008F939F93AF93BF93EF93FF938091E100A9
:1019500082FF0BC08091E20082FF07C08091E1000E
:101960008B7F8093E1000E94FC0E8091DA0080FF63
:101970001FC08091D80080FF1BC08091DA008E7F4D
:101980008093DA008091D90080FF0DC080E189BD8D
:1019900082E189BD09B400FEFDCF81E08093F101B1
:1019A0000E94F70805C019BC1092F1010E940509B8
:1019B0008091E10080FF19C08091E20080FF15C096
:1019C0008091E2008E7F8093E2008091E20080614E
:1019D0008093E2008091D80080628093D80019BC87
:1019E00085E08093F1010E9409098091E10084FF64
:1019F00030C08091E20084FF2CC080E189BD82E18B
:101A000089BD09B400FEFDCF8091D8008F7D809301
:101A1000D8008091E1008F7E8093E1008091E20008
:101A20008F7E8093E2008091E20081608093E200EB
:101A30008091ED01882311F084E007C08091E300DC
:101A400087FD02C081E001C083E08093F1010E9424
:101A50000B098091E10083FF29C08091E20083FFA0
:101A600025C08091E100877F8093E10082E0809330
:101A7000F1011092ED018091E1008E7F8093E100F1
:101A80008091E2008E7F8093E2008091E20080618D
:101A90008093E20042E060E080E00E94940B80913D
:101AA000F00088608093F0000E940809FF91EF9198
:101AB000BF91AF919F918F917F916F915F914F9166
:101AC0003F912F910F900FBE0F901F9018951F926E
:101AD0000F920FB60F9211242F933F934F935F9362
:101AE0006F937F938F939F93AF93BF93CF93DF9326
:101AF000EF93FF93C091E900CF708091EC00D82F55
:101B0000D17080FDD0E81092E9008091F000877FCD
:101B10008093F00078940E94AB0D1092E9008091C0
:101B2000F00088608093F000CD2BCF70C093E90067
:101B3000FF91EF91DF91CF91BF91AF919F918F91E5
:101B40007F916F915F914F913F912F910F900FBEB9
:101B50000F901F9018951F93CF93DF93CDB7DEB7EB
:101B6000AA970FB6F894DEBF0FBECDBFE2EFF1E04B
:101B700088E08E0F9091F10091938E13FBCF0E941D
:101B800027098091E80083FF1FC18091F2019091A5
:101B9000F301492F50E04A30510508F015C1FA0110
:101BA000EA5AFF4F0C949622803881F0823809F06F
:101BB0000BC18091F6018F708093E9008091EB005A
:101BC00085FB882780F91092E90006C08091EE011C
:101BD0009091EF01911182609091E800977F90932E
:101BE000E8008093F1001092F100C8C0282F2D7FEB
:101BF00009F0EAC0882319F0823061F0E5C08091D5
:101C0000F401813009F0E0C0933009F080E0809366
:101C1000EF012BC08091F401811127C08091F60162
:101C20008F7009F4D1C08093E9002091EB0020FF70
:101C30001CC0933021F48091EB00806214C090911D
:101C4000EB0090619093EB0021E030E0A90102C02D
:101C5000440F551F8A95E2F74093EA001092EA007C
:101C60008091EB0088608093EB001092E9008091F6
:101C7000E800877F86C08111A7C01091F4011F770B
:101C80008091E3008078812B8093E3008091E800CD
:101C9000877F8093E8000E94C90B8091E80080FF55
:101CA000FCCF8091E30080688093E300111102C0B3
:101CB00082E001C083E08093F10186C080588230C9
:101CC00008F082C08091F4019091F5018C3D53E0C1
:101CD000950779F583E08A838AE289834FB7F89480
:101CE000DE01139620E03EE051E2E32FF0E0509356
:101CF0005700E49120FF03C0E295EF703F5FEF7063
:101D00008E2F90E0EA3010F0C79601C0C0968D93F8
:101D10009D932F5F243149F74FBF8091E800877F63
:101D20008093E8006AE270E0CE0101960E94D00A3A
:101D300014C0AE014F5F5F4F6091F6010E94170A19
:101D4000BC01009709F440C09091E800977F909300
:101D5000E80089819A810E94330B8091E8008B779B
:101D60008093E80031C0803879F58091E800877F62
:101D70008093E8008091ED018093F1008091E8006C
:101D80008E778093E8000E94C90B1EC081111CC091
:101D90009091F4019230C0F48091E800877F8093A5
:101DA000E8009093ED010E94C90B8091ED01811133
:101DB00006C08091E30087FD02C081E001C084E09D
:101DC0008093F1010E9413098091E80083FF0AC00B
:101DD0008091E800877F8093E8008091EB0080622B
:101DE0008093EB00AA960FB6F894DEBF0FBECDBF6E
:101DF000DF91CF911F9108950895CF938091F101C4
:101E00008823A1F0C091E900CF709091EC00892F58
:101E1000817090FD80E8C82B1092E9008091E80065
:101E200083FD0E94AB0DCF70C093E900CF91089560
:101E300090937501809374010895E0917401F0917D
:101E40007501309721F00190F081E02D099480E038
:101E50000895E0917401F0917501309721F00280AE
:101E6000F381E02D09940895E0917401F0917501DA
:101E7000309721F00480F581E02D09940895209198
:101E80007201309173018217930771F0909373017F
:101E900080937201E0917401F0917501309721F007
:101EA0000680F781E02D099408952091700130910A
:101EB00071018217930771F0909371018093700103
:101EC000E0917401F0917501309721F00084F18563
:101ED000E02D0994089508950C946B0F0E94751AD3
:101EE0000E9489020C94371B9F92AF92BF92CF92AF
:101EF000DF92EF92FF920F931F93CF93DF9300D067
:101F000000D000D0CDB7DEB70E94A1020DE010E0F6
:101F1000AA24A394B12C902E802F0E948F039801A5
:101F200029583E4F6901F901F080F826A1F40150CB
:101F3000110988F78FEF89838A831B820E947E1A9A
:101F40008160782F9D838C8349815A816B818D813B
:101F50000E940B102FC09091DA0191FF04C08E8374
:101F60000E9495038E8125E030E0A501022E01C07C
:101F7000440F0A94EAF7E42E4F21C1F029839A8294
:101F80008E2191E009F490E09B830E947E1A81608B
:101F9000782F9D838C8349815A816B818D810E942A
:101FA0000B10F6018081E826E08204C0215031093F
:101FB000E0F6BDCF0E941E1E109176010E941D0FFB
:101FC0001817B9F00E941D0F8093760126960FB660
:101FD000F894DEBF0FBECDBFDF91CF911F910F915F
:101FE000FF90EF90DF90CF90BF90AF909F900C94B8
:101FF000160826960FB6F894DEBF0FBECDBFDF9150
:10200000CF911F910F91FF90EF90DF90CF90BF90F5
:10201000AF909F900895CF93DF93CDB7DEB72B9706
:102020000FB6F894DEBF0FBECDBF4F8358876987C8
:102030007A878B87DE01119686E0FD0111928A95E1
:10204000E9F785E0FE01379601900D928A95E1F758
:1020500049815A816B817C818D819E810E945416B9
:102060002B960FB6F894DEBF0FBECDBFDF91CF9198
:102070000895CF93882309F4C2C0C82F823859F439
:102080000E941D0F81FDBBC089E30E942E190E9492
:10209000FB1989E30CC0833879F40E941D0F80FD81
:1020A000AEC083E50E942E190E94FB1983E50E94B1
:1020B0007019CF910C94FB19843859F40E941D0FAC
:1020C00082FD9DC087E40E942E190E94FB1987E4BF
:1020D000EECF8CEF8C0F813A48F48C2F0E94612058
:1020E00081118DC08C2F0E942E19E3CF80E28C0FBE
:1020F000883048F4C77081E001C0880FCA95EAF7BC
:102100000E94B419D6CF8BE58C0F833078F4C53A92
:1021100029F0C63A31F083E890E005C081E890E00C
:1021200002C082E890E0CF910C943F0F88E58C0FBD
:10213000833108F064C0C83A39F1C93A41F1CA3A6A
:1021400049F1CB3A51F1CC3A59F1CD3A61F1C03B6A
:1021500069F1CE3A71F1CF3A79F1C13B81F1C23BDD
:1021600089F1C33B91F1C43B99F1C53BA1F1C63B59
:10217000A9F1C73BB1F1C83BB9F1C93BC1F1CA3BB9
:10218000C9F180E090E038C082EE90E035C089EE81
:1021900090E032C08AEE90E02FC085EB90E02CC03A
:1021A00086EB90E029C087EB90E026C08CEC90E0B5
:1021B00023C08DEC90E020C083E891E01DC08AE848
:1021C00091E01AC082E991E017C084E991E014C05F
:1021D00081E292E011C083E292E00EC084E292E0DC
:1021E0000BC085E292E008C086E292E005C087E27B
:1021F00092E002C08AE292E0CF910C94550FCF9109
:102200000895882309F44BC0823859F40E941D0FA9
:1022100081FF45C089E30E942E190E94FB1989E3C2
:102220000CC0833871F40E941D0F80FF38C083E515
:102230000E942E190E94FB1983E50E9470190C94CC
:10224000FB19843859F40E941D0F82FF28C087E4CF
:102250000E942E190E94FB1987E4EFCF9CEF980F84
:10226000913A58F390E2980F983050F4877091E0CB
:1022700001C0990F8A95EAF7892F0E94BA19DFCF1A
:102280009BE5980F933020F480E090E00C943F0F92
:10229000885A833120F480E090E00C94550F089523
:1022A000882321F00E94B4190C94FB190895882307
:1022B00021F00E94BA190C94FB1908957F928F9215
:1022C0009F92AF92BF92CF92DF92EF92FF920F93C5
:1022D0001F93CF93DF931F92CDB7DEB77C01C62E3D
:1022E000772EFC01058102950F70128111110E9459
:1022F000D1190E942719882379F0112369F080E20F
:102300008C0D883048F082E00E9410190E94271935
:1023100091E0D82ED92601C0D12CE72DE295EF709F
:10232000F0E0E05AFF4F0C949622872D807F072D16
:102330000F70882311F00295007F112389F000238C
:1023400009F490C180E28C0D883020F4802F0E9427
:10235000B41903C0802F0E94C4190E94FB1982C1C6
:102360008C2D0E940111002309F495C180E28C0D8F
:10237000883020F4802F0E94BA1903C0802F0E9459
:10238000CA190E94FB1987C1972D907F872D8F70E6
:10239000903211F08295807FCC2021F0F1E0CF16B1
:1023A000B1F01EC0112349F0002309F414C101301B
:1023B00009F011C10E94E4196EC1002319F0013027
:1023C00009F469C189830E94E71989810AC111232F
:1023D00021F0023008F05FC1FEC001115CC101C1F3
:1023E000112321F0002309F4F6C03CC1002309F4B5
:1023F000F8C03EC1872D86958695837090E0009742
:1024000019F0019761F047C1112321F08C2D972D10
:10241000937002C080E090E00E943F0F3CC1112306
:1024200021F08C2D972D937002C080E090E00E94E7
:10243000550F31C18C2D112319F00E94261D02C0A9
:102440000E948E1D0E94131E26C1872D837009F0E5
:1024500052C0111120C18C2D829586958770880FEE
:10246000880F9C2D9F70892E912CA12CB12C082EA9
:1024700004C0880C991CAA1CBB1C0A94D2F7C4FE89
:1024800014C00FE010E020E030E0B901A80104C062
:10249000440F551F661F771F8A95D2F7CB01BA01EB
:1024A000609570958095909503C060E070E0CB01D9
:1024B000272D26952695237030E02230310569F0CE
:1024C0002330310589F0682979298A299B2921300F
:1024D000310571F00E949C17DEC0682979298A298C
:1024E0009B290E94B817D7C00E949C17C501B40150
:1024F0000E948017D0C0112319F0872D817001C070
:102500008695882309F4C7C08C2D8295869587709F
:10251000880F880F9C2D9F70892E912CA12CB12C97
:10252000082E04C0880C991CAA1CBB1C0A94D2F764
:10253000C4FE14C00FE010E020E030E0B901A801B3
:1025400004C0440F551F661F771F8A95D2F7CB0131
:10255000BA01609570958095909503C060E070E039
:10256000CB01272D269526952370422F50E042302F
:10257000510569F04330510589F0682979298A2984
:102580009B294130510571F00E94761884C068295A
:1025900079298A299B290E9492187DC00E94761869
:1025A000C501B4010E945A1876C08C2D90E0FC0140
:1025B000E05EF109E531F10508F050C0E059FF4F48
:1025C0000C9496220C2D0F70872D8F71112331F0F2
:1025D0000E94F317802F0E9450115DC00E941418B2
:1025E000802F0E94571157C0112339F0011153C099
:1025F000872D8F710E9439184EC0023008F04BC0F1
:10260000F7CF112339F0872D8F710E94F31743C044
:102610001123C9F3872D8F710E9414183CC0112318
:1026200029F0872D8F710E94DE1735C00E94D417C4
:1026300032C0112351F0172D1F71812F0E94F31703
:1026400063E0812F0E94071926C081E00E941019C3
:10265000023008F182E00E9410191DC0112331F0F0
:10266000002389F28C2D0E94391015C0002391F2AD
:102670008C2D0E9401110FC0472D4F706C2DC7018A
:102680000E946B040E94F81606C0472D4F706C2DF7
:10269000C7010E942505DD20F9F00E94031980FD85
:1026A0001BC0F70112820E94FD180E94F317C70198
:1026B0000E947B130E94FD180F90DF91CF911F9114
:1026C0000F91FF90EF90DF90CF90BF90AF909F90D1
:1026D0008F907F900C9414180F90DF91CF911F91E1
:1026E0000F91FF90EF90DF90CF90BF90AF909F90B1
:1026F0008F907F9008950F931F93CF93DF93EC01FA
:10270000888199812B813C81232BB9F09F3F11F463
:102710008F3F99F0CE010E947D04882371F068817B
:1027200079818A810E94F9188C010E94AE180E945A
:102730007517B801CE010E945E11DF91CF911F91F4
:102740000F9108950E94D1190E94E1190E94A619C3
:102750000E94FB190E94C41E0E94131E80E090E09C
:102760000E943F0F80E090E00C94550F0E94C11929
:102770000C94A2130E94EE18292F22952F7030E09E
:102780002C3031054CF42A3031056CF422503109DB
:1027900022303105A8F407C02C30310569F02F3004
:1027A000310551F00DC0803F69F018F4803E40F4CF
:1027B00009C0843F29F406C093FB882780F9089557
:1027C00080E0089581E00895CF93DF9300D000D09A
:1027D0001F92CDB7DEB70F900F900F900F900F9014
:1027E000DF91CF910895CF93DF9300D000D000D038
:1027F000CDB7DEB726960FB6F894DEBF0FBECDBFBD
:10280000DF91CF9108951F93CF93DF93C0918501FE
:1028100016E080918601C81799F0D0E01C9FF00166
:102820001D9FF00D1124E957FE4F408151816281B7
:102830007381848195810E94F3132196C770E9CF3B
:10284000DF91CF911F9108954091B7015091B80148
:102850006091B9017091BA018091BB019091BC0166
:102860000C94F3138091BC0182958F7009F054C0D1
:102870008091B901882309F44FC080918501A0910E
:1028800086016091B7017091B8014091BA015091F1
:10289000BB01B6E08A1709F43FC090E0411551052D
:1028A000C1F17F3F11F46F3FA1F1B89FF001B99FD3
:1028B000F00D1124E957FE4F218172132AC02081A7
:1028C000621327C02281211124C02381348124175F
:1028D000350710F421503109241B350B283C3105F4
:1028E000C0F42091BC012F7020612093BC0126E030
:1028F000289FF001299FF00D1124E457FE4F80819D
:102900008F708061808387EB91E00E947B130C9431
:10291000031401968770BECF0895CF92DF92EF9295
:10292000FF920F931F93CF93DF93CDB7DEB76297DC
:102930000FB6F894DEBF0FBECDBF8C0185E0F80165
:10294000DE011D9601900D928A95E1F7D8014C9118
:1029500011965C91119712966C9112971396CD90E7
:10296000DC9014973091B7017091B8018091BA0151
:102970009091BB01009709F46BC17F3F19F43F3F71
:1029800009F466C1E090B901EE2009F4C0C02091BD
:10299000BC01C816D90628F0F601E81BF90BCF01D7
:1029A00004C0809590958C0D9D1DFF24F394883C68
:1029B000910578F0F12C207F09F0C6C07C2DD98AD2
:1029C000C88A89890E94E41387EB91E00E947B13F7
:1029D000B1C0822F807F09F046C0751314C0341334
:1029E00012C0611110C02F7020612093BC010E94A1
:1029F000241487EB91E00E947B138091BC01D801E5
:102A000015968C932EC0CD2819F15F3F11F44F3FDE
:102A1000F9F0F62E61111CC080918501209186018C
:102A200036E0821709F45AC090E0389FF001399FD0
:102A3000F00D1124E957FE4F7181571306C07081C4
:102A4000471303C07281711103C001968770E9CFEB
:102A5000F62E662309F418C18091BC018160809331
:102A6000BC01F12C11C1751308C0341306C06111EB
:102A700004C08091BC01D801C3C04D875E878D859D
:102A80009E856A8B0E94BA136A898823E1F16623C6
:102A9000D1F12091BC01822F82958F7090E0029736
:102AA00074F08091B7019091B80198878F8319864F
:102AB000DB86CA862C87CE0107960E947B1386E0B0
:102AC000F801A7EBB1E001900D928A95E1F70E9421
:102AD00032140E942414FF24F394D6C04D875E87DD
:102AE0008D859E850E94EE18292F22952F7030E04B
:102AF000223031050CF0BCC09F7009F0B6C0805E7A
:102B0000883008F4C1C0C8010E947B13E4CFC81606
:102B1000D90608F453C0F601E81BF90BCF01883C35
:102B2000910508F450C0F12C7C2DD98AC88A898976
:102B30000E94E413E7EBF1E086E0DF011D928A9545
:102B4000E9F70E942414A0C0751314C0341312C0F6
:102B5000611110C08091BC01F8018583C8010E94F9
:102B60007B1386E0E7EBF1E0DF011D928A95E9F740
:102B7000FE2C8AC04D875E878D859E856A8B0E945C
:102B8000BA136A89882309F4BECF662309F4BBCF40
:102B90002091BC01822F82958F7090E002970CF4F7
:102BA0008ECF8091B7019091B8019A8389831B825F
:102BB000DD82CC822E83CE0101967FCF80959095C9
:102BC0008C0D9D1DACCFF62E662309F49CCF75139A
:102BD0002EC034132CC02091BC0120FD1FC0822FB9
:102BE00082958F70D9F0D80115962C9315978F3058
:102BF00049F08F5F982F9295907F822F8F70892B4D
:102C000015968C93C8010E947B1386E0F801A7EB10
:102C1000B1E001900D928A95E1F793CF86E0F8013B
:102C2000A7EBB1E001900D928A95E1F72DC04D8799
:102C30005E878D859E850E94BA13811140CF809159
:102C4000BC0181608093BC01C8010E947B131CC041
:102C5000662309F458CF4D875E878D859E850E9437
:102C6000BA13882309F44FCF2ACF811148CF0CC063
:102C7000243031050CF047CF9F7009F440CFF801A4
:102C80009581907F09F03BCF8F2D62960FB6F89417
:102C9000DEBF0FBECDBFDF91CF911F910F91FF908F
:102CA000EF90DF90CF9008951F93CF93DF93CDB730
:102CB000DEB72C970FB6F894DEBF0FBECDBF4F83A3
:102CC000588769877A878B879C87CE0107960E94F1
:102CD0008D14882369F08F8198852A853B85232B65
:102CE000F1F19F3F09F063C08F3F09F060C037C02A
:102CF00086E0FE013796DE01119601900D928A95CD
:102D0000E1F76F817885EA85FB85309741F17F3F58
:102D100011F46F3F21F12091860130E0C901019645
:102D2000877099274091850150E08417950709F431
:102D300047C069837A83FD83EC8396E0929FD0013C
:102D4000939FB00D1124A957BE4FFE0131960190FB
:102D50000D929A95E1F7809386010E94031416E084
:102D600080918501909186018917C1F1189FC0015A
:102D7000112489579E4F0E948D14882379F1E09188
:102D800085011E9FF0011124E957FE4F40815181BA
:102D900062817381848195810E94F3138091850102
:102DA00090E001968770992780938501D9CF4F8154
:102DB000588569857A858B859C850E94F313CFCFD2
:102DC0000E94B6131092860110928501E7EBF1E0A4
:102DD00086E0DF011D928A95E9F7C1CF2C960FB6E8
:102DE000F894DEBF0FBECDBFDF91CF911F91089544
:102DF000EF92FF920F931F93CF93DF938C01009775
:102E000009F46CC0F12CEE24E394E8012196F8015A
:102E10008491843740F4843008F051C0813081F0CF
:102E2000823019F15BC0853709F444C0A8F19CE7F2
:102E3000980F903708F052C08F770E94011141C05F
:102E40000E5F1F4FFE01C49180E28C0F883048F462
:102E5000C7708E2D01C0880FCA95EAF70E94D41959
:102E600014C08C2F0E9439102DC00E5F1F4FFE0121
:102E7000C49180E28C0F883058F4C7708E2D01C049
:102E8000880FCA95EAF70E94DA190E94FB191AC046
:102E90008C2F0E94011116C00E5F1F4FFE01C491BE
:102EA000CC2381F08FE99FE00197F1F700C000008B
:102EB000C150F6CF0E5F1F4FFE01F49003C00E9479
:102EC00039108E018F2D882309F49FCFEFE9FFE0A1
:102ED0003197F1F700C000008150F5CFDF91CF911D
:102EE0001F910F91FF90EF90089508956093C10195
:102EF0007093C2018093C3019093C4010C94A213F8
:102F00000F931F930091C1011091C2012091C30141
:102F10003091C401DC01CB01802B912BA22BB32B70
:102F20008093C1019093C201A093C301B093C401E7
:102F30001F910F910C94A2130F931F930091C10145
:102F40001091C2012091C3013091C401DC01CB0179
:102F500080239123A223B3238093C1019093C201C4
:102F6000A093C301B093C4011F910F910C94A213BD
:102F70000F931F930091C1011091C2012091C301D1
:102F80003091C401DC01CB0180279127A227B32710
:102F90008093C1019093C201A093C301B093C40177
:102FA0001F910F910C94A2131092BD011092BE01BB
:102FB0001092BF011092C0010C94A21341E050E0A6
:102FC00060E070E004C0440F551F661F771F8A95AC
:102FD000D2F74093BD015093BE016093BF0170933F
:102FE000C0010C94A21341E050E060E070E004C026
:102FF000440F551F661F771F8A95D2F78091BD0138
:103000009091BE01A091BF01B091C001482B592BF6
:103010006A2B7B2B4093BD015093BE016093BF018F
:103020007093C0010C94A21341E050E060E070E0A6
:1030300004C0440F551F661F771F8A95D2F740952D
:103040005095609570958091BD019091BE01A091C1
:10305000BF01B091C001482359236A237B234093C9
:10306000BD015093BE016093BF017093C0010C94E9
:10307000A21341E050E060E070E004C0440F551F2F
:10308000661F771F8A95D2F78091BD019091BE018E
:10309000A091BF01B091C001482759276A277B271B
:1030A0004093BD015093BE016093BF017093C00176
:1030B0000C94A2130F931F930091BD011091BE01B8
:1030C0002091BF013091C001DC01CB01802B912BFD
:1030D000A22BB32B8093BD019093BE01A093BF019F
:1030E000B093C0011F910F910C94A2130F931F93E3
:1030F0000091BD011091BE012091BF013091C0012E
:10310000DC01CB0180239123A223B3238093BD0153
:103110009093BE01A093BF01B093C0011F910F9186
:103120000C94A2130F931F930091BD011091BE0147
:103130002091BF013091C001DC01CB018027912794
:10314000A227B3278093BD019093BE01A093BF0136
:10315000B093C0011F910F910C94A2130895CF92C8
:10316000DF92EF92FF920F931F93CF93DF938C0127
:10317000C090C101D090C201E090C301F090C401A1
:103180008091BD019091BE01A091BF01B091C0019D
:10319000C82AD92AEA2AFB2ACFE1D0E0D701C60102
:1031A0000C2E04C0B695A795979587950A94D2F7EB
:1031B00080FF06C0B8018C2F0E947B07019721F485
:1031C000219760F780E001C08C2FDF91CF911F9194
:1031D0000F91FF90EF90DF90CF900895CF93DF9302
:1031E000EC010E94AF18BE010E947B07DF91CF91D6
:1031F0000895CB010E94EE1808958091C501859530
:103200008595859508958091C5018770089598E00A
:10321000899F90011124262B2093C5010C94F3174C
:103220002091C501809582238093C501982F9770C6
:1032300069F430E0482F552747FD5095241735078E
:1032400029F08595859585950C941418089590918D
:10325000C501977081E009F480E0089590910C0118
:10326000992321F090910D01911109C020910E0137
:1032700030910F01F90132969FEF40E01FC0982F67
:103280009695969596959F3050F5E0910E01F091A8
:103290000F01E90FF11D877021E030E0A90102C0A4
:1032A000440F551F8A95E2F7CA019181892B8183CA
:1032B00008959F3F39F04F5F4E3041F051915813C0
:1032C000F8CF0DC05111F7CF942FF5CF9F3F39F0B4
:1032D000F901E90FF11D97FDFA958283089508958C
:1032E00090910C01992321F090910D01911109C049
:1032F00020910E0130910F01F9013296205F3F4F6E
:103300001FC0982F9695969596959F30F0F4E09172
:103310000E01F0910F01E90FF11D877021E030E0FF
:10332000A90102C0440F551F8A95E2F7CA01809592
:1033300091818923818308953196E217F30729F05B
:1033400090819813F9CF1082F7CF089581E090E033
:10335000E0910E01F0910F01E80FF91F1082019624
:1033600080319105A9F708959091D901892B809317
:10337000D901089580959091D90189238093D9012D
:1033800008951092D90108959091D801892B8093C6
:10339000D801089580959091D80189238093D80110
:1033A00008951092D80108959091D701892B8093A8
:1033B000D701089580959091D70189238093D701F3
:1033C00008951092D70108958093C6010895109230
:1033D000C601089580910E0190910F01FC01319674
:1033E0009C01205F3F4F80E0919191118F5FE21728
:1033F000F307D1F70895E0910E01F0910F0180914C
:10340000D9018083E0910E01F0910F0190818091AC
:10341000D801892B8083E0910E01F0910F019081FA
:103420008091D701892B80838091C601882361F028
:10343000E0910E01F0910F019081892B80830E9411
:10344000EA1981111092C60180910E0190910F012D
:103450000C94290F20E0009739F0AC01415051093C
:10346000842395232F5FF7CF822F08958091F10158
:10347000843021F11092DB0120E488E190E00FB666
:10348000F894A895809360000FBE2093600080E0C0
:103490000E94160883B7817F846083BF83B78160F1
:1034A00083BF7894889583B78E7F83BF88E10FB6FA
:1034B000F89480936000109260000FBE0895089504
:1034C00008950E945F1A0E94A1020E94601A0E9441
:1034D000960391E0811101C090E0892F08950E9428
:1034E000B6130E941D0F0C94160882E084BD93E071
:1034F00095BD9AEF97BD80936E0008952FB7F8940D
:103500008091DC019091DD01A091DE01B091DF019D
:103510002FBF0895CF92DF92EF92FF920F931F93E8
:103520002FB7F8944091DC015091DD016091DE01EC
:103530007091DF012FBF6A017B01EE24FF248C0113
:1035400020E030E0C016D106E206F30610F4415048
:1035500051099A01281B390BC9011F910F91FF9046
:10356000EF90DF90CF9008951F920F920FB60F92B9
:1035700011248F939F93AF93BF938091DC0190911F
:10358000DD01A091DE01B091DF010196A11DB11D09
:103590008093DC019093DD01A093DE01B093DF0105
:1035A000BF91AF919F918F910F900FBE0F901F9081
:1035B00018950E941A0CF8942FEF87EA91E6215093
:1035C00080409040E1F700C0000087E090EBDC0114
:1035D0008093FB019093FC01A093FD01B093FE0149
:1035E0009CE088E10FB6F894A895809360000FBE28
:1035F00090936000FFCFEF92FF920F931F93CF93B2
:10360000DF93D82FCDE08C2F0E948F0305E010E0D0
:10361000E82EF12CC701002E02C0959587950A94DB
:10362000E2F780FF09C0602F7C2F80E00E94260512
:10363000D81302C081E006C00150110958F7C150EB
:1036400010F780E0DF91CF911F910F91FF90EF90E5
:103650000895CF93C82F8CE20E94FB1A882321F093
:103660008C2FCF910C94FB1A80E0CF910895CF93CB
:103670000E947E1C811102C00E94641CC5E6C150DC
:1036800049F00E94A1028FE39CE90197F1F700C085
:103690000000F5CF89E20E94291B811113C18AE243
:1036A0000E94291B81110E94641C85E00E94291B35
:1036B00081110E94D91A0E94891C8093DA0187E047
:1036C0000E94291B8823A9F18BE10E94291B8823D2
:1036D00051F08091DA0181FB222720F991E09227B5
:1036E00090FB81F90EC08EE00E94291B882361F0B7
:1036F0008091DA0182FB222720F991E0922790FB4A
:1037000082F98093DA0115C080E10E94291B909113
:10371000DA01882341F093FB222720F981E08227F8
:1037200080FB93F904C0892F809580FB90F99093DA
:10373000DA018091DA010E948D1C0E949B1C80930B
:10374000FA0180EE0E94291B882341F08091FA0142
:10375000982F909590FB80F98093FA0189E30E945D
:10376000291B882359F08091FA0181FB222720F937
:1037700091E0922790FB81F98093FA0182EE0E94FA
:10378000291B882359F08091FA0182FB222720F916
:1037900091E0922790FB82F98093FA0186EE0E94D5
:1037A000291B882359F08091FA0183FB222720F9F5
:1037B00091E0922790FB83F98093FA0183EE0E94B7
:1037C000291B882359F08091FA0184FB222720F9D4
:1037D00091E0922790FB84F98093FA0185E30E949F
:1037E000291B882359F08091FA0185FB222720F9B3
:1037F00091E0922790FB85F98093FA0181E30E9482
:10380000291B882359F08091FA0186FB222720F991
:1038100091E0922790FB86F98093FA0181E10E9462
:10382000291B882359F08091FA0187FB222720F970
:1038300091E0922790FB87F98093FA018091FA0139
:103840000E949F1C8091FA0187FB882780F9809352
:103850000D0187E20E94291BC82F8EE10E94291BBF
:103860008111C2608FE10E94291B8111C46080E236
:103870000E94291B8111C86081E20E94291B8111CD
:10388000C06182E20E94291B8111C06283E20E9412
:10389000291B8111C06484E20E94291B882311F036
:1038A000C06802C0CC2329F08C2F0E94961C6C2F7C
:1038B00003C00E94921C682F70E080E090E0CF91DE
:1038C0000C947617CF9108956DEE7EEF80E090E036
:1038D0000E94D02260E082E090E00E94BE2260E080
:1038E00083E090E00E94BE2260E084E090E00E94CD
:1038F000BE2260E085E090E00C94BE2280E090E083
:103900000E94B82221E08D3E9E4F09F020E0822FD8
:10391000089582E090E00C94B022682F82E090E05D
:103920000C94BE2283E090E00C94B022682F83E0D8
:1039300090E00C94BE2284E090E00C94B022682FBA
:1039400084E090E00C94BE228091E20180FF0BC0E5
:103950006091130185E0689FB0011124759567950A
:10396000759567952BC081FF09C06091130185E0B3
:10397000689FB00111247595679520C082FF07C02C
:103980006091130185E0689FB001112417C09091E8
:10399000E3019923D1F060911201961788F72091E5
:1039A000130185E0289F90011124929FA001939F0D
:1039B000500D112470E0CA010E9482226038710506
:1039C00040F46115710539F002C065E070E0862FA2
:1039D00008958FE7089581E008958091E20180FFC6
:1039E00008C06091110170E07595679575956795B0
:1039F00021C081FF06C06091110170E07595679547
:103A000019C082FF04C06091110170E010C0909154
:103A1000E3019923C1F0609110019617A0F78091FE
:103A20001101899FC001112470E00E948222603838
:103A3000710528F46115710521F0862F08958FE72F
:103A4000089581E0089561E070E0F4CF803F21F4B3
:103A50000E94A41C819504C0813F29F40E94A41CEB
:103A60008093E6010895823F21F40E94A41C819571
:103A700004C0833F29F40E94A41C8093E5010895AB
:103A8000893F19F40E94ED1C05C08A3F31F40E9461
:103A9000ED1C81958093E70108958B3F21F40E94EE
:103AA000ED1C819504C08C3F29F40E94ED1C80938D
:103AB000E8010895843F21F48091E401816017C0FA
:103AC000853F21F48091E401826011C0863F21F49A
:103AD0008091E40184600BC0873F21F48091E40170
:103AE000886005C0883F31F48091E4018061809353
:103AF000E40108958D3F21F48091E20181600BC0C3
:103B00008E3F21F48091E201826005C08F3F29F44D
:103B10008091E20184608093E2010895803F39F44E
:103B20008091E60187FF6CC01092E60169C0813F79
:103B300029F48091E6011816BCF362C09091E5016A
:103B4000823F29F497FF5CC01092E50159C0833F82
:103B500019F41916CCF354C0893F41F48091E70160
:103B600018160CF04DC01092E7014AC08A3F29F4A4
:103B70008091E70187FF44C0F6CF8B3F39F48091F5
:103B8000E80187FF3DC01092E8013AC08C3F29F45C
:103B90008091E8011816BCF333C0843F21F4809172
:103BA000E4018E7F17C0853F21F48091E4018D7F71
:103BB00011C0863F21F48091E4018B7F0BC0873FC9
:103BC00021F48091E401877F05C0883F31F4809122
:103BD000E4018F7E8093E40113C08D3F21F4809136
:103BE000E2018E7F0BC08E3F21F48091E2018D7F38
:103BF00005C08F3F29F48091E2018B7F8093E20121
:103C00008091E50181110EC08091E60181110AC009
:103C10008091E701811106C08091E801811102C005
:103C20001092E301089584EE91E00E94340F0E9407
:103C30007E1A9093E1018093E00108951F93CF9342
:103C4000DF938091E0019091E1010E948A1AAC011A
:103C50009091E301992321F02091140130E006C0F6
:103C6000209115018AE0289F9001112442175307E3
:103C700008F486C08091E501C091E601D091E7018A
:103C80001091E801811107C0C11176C0D11174C033
:103C9000111172C075C09F3F19F09F5F9093E301AF
:103CA000181624F40E94A41C8093E5018091E5017C
:103CB00087FF05C00E94A41C81958093E5011C1616
:103CC00024F40E94A41C8093E6018091E60187FF02
:103CD00005C00E94A41C81958093E6016091E501D6
:103CE000662339F1C091E601CC2319F1772767FDEE
:103CF0007095872F972F0E94932123E333E343E3AB
:103D00005FE30E94F7210E9460216093E5016C2F20
:103D1000772767FD7095872F972F0E94932123E3C4
:103D200033E343E35FE30E94F7210E946021609345
:103D3000E6011D1624F40E94ED1C8093E70180919A
:103D4000E70187FF05C00E94ED1C81958093E70184
:103D5000111624F40E94ED1C8093E8018091E80183
:103D600087FF05C00E94ED1C81958093E801DF91DB
:103D7000CF911F910C94131E9F3F09F08ECF96CFC9
:103D8000DF91CF911F910895E4EEF1E085E0DF012E
:103D90001D928A95E9F71092E3011092E2010895CD
:103DA000833081F128F4813059F08230D1F00895C8
:103DB000853009F449C0B8F1863009F456C0089539
:103DC00080911501262F30E0280F311D2F3F31053E
:103DD00024F4680F6093150108958FEF8093150107
:103DE000089580911401262F30E0280F311D2F3FB8
:103DF000310524F4680F6093140108958FEF8093C8
:103E00001401089580911301262F30E0280F311DF1
:103E10002F3F310524F4680F6093130108958FEF4D
:103E200080931301089580911201262F30E0280F0E
:103E3000311D2F3F310524F4680F6093120108955E
:103E40008FEF80931201089580911101262F30E0A9
:103E5000280F311D2F3F310524F4680F60931101A5
:103E600008958FEF80931101089580911001262FFE
:103E700030E0280F311D2F3F310524F4680F609387
:103E8000100108958FEF809310010895833011F190
:103E900028F4813049F0823091F00895853081F125
:103EA00020F18630C1F1089580911501681720F442
:103EB000861B809315010895109215010895809135
:103EC0001401681720F4861B809314010895109242
:103ED0001401089580911301681720F4861B8093C4
:103EE000130108951092130108958091120168172B
:103EF00020F4861B809312010895109212010895F8
:103F000080911101681720F4861B80931101089598
:103F100010921101089580911001681720F4861BFA
:103F20008093100108951092100108950F931F932C
:103F30008D3109F46BC008F03FC08E3009F47FC0AA
:103F4000C0F4873009F469C068F4863009F0B1C064
:103F50008091DA01817F8E7F8093DA0181E0809306
:103F6000EA01A8C0883009F4A2C08B3009F49FC0D0
:103F7000A0C0863109F49BC078F4803109F472C086
:103F8000813109F096C00E94B61390910D0181E035
:103F9000892780930D018BC0893109F488C08B314A
:103FA00009F087C08091DA0181FB222720F991E096
:103FB000922790FB81F94CC0853309F470C048F416
:103FC000873209F46CC008F459C0893209F467C01B
:103FD00070C0833438F48A3308F04EC0883309F453
:103FE00066C067C0833409F45AC0883409F061C0E0
:103FF0000E94B6130FEF13ED20E301501040204054
:10400000E1F700C000000E94D91A51C00E941A2195
:104010000E941D0F0E9416084AC09091DA01892F54
:104020008095817080FB90F929F09660986090935C
:10403000DA0140C0997F977F9093DA0138C0809170
:10404000DA0182FB222720F991E0922790FB82F986
:104050008093DA01992359F18091DA01816080938C
:10406000DA0125C08091DA0183FB222720F991E053
:10407000922790FB83F9ECCF895301C08D5141E029
:1040800050E060E070E08A019B0104C0000F111F46
:10409000221F331F8A95D2F7C901B80104C061E01D
:1040A00070E080E090E00E9476170E94B61381E0F5
:1040B00001C080E01F910F91089580E0089580E095
:1040C0000895CF93C82F8091EA01813079F018F0DC
:1040D0008230E9F187C0E0910E01F0910F018081FB
:1040E000813169F0823209F07FC009C0E0910E0190
:1040F000F0910F018081813111F0823261F48C2FB7
:104100000E945D20811104C08C2F0E94961F1DC04B
:1041100081E090E01AC08C2F0E945F20811114C0B2
:10412000C43179F048F4CB3079F0C03109F060C087
:1041300082E08093EA0108C0C93219F0C83321F047
:1041400057C01092EA0154C081E0817053C0C93257
:1041500089F118F5C43171F1A8F4C73009F046C0EF
:104160008AE08093150194E19093140193E0909379
:1041700013018093120188E08093110188E28093FB
:10418000100134C0CE51C63088F5EC2FF0E0E65D6A
:10419000FE4F80818093E90129C0CE34E9F020F4FC
:1041A000CB3421F56AE013C0C13579F0C235F1F4A2
:1041B00061E00DC08091E901882319F01092E901B6
:1041C00015C081E08093EA0115C061E006C08091CE
:1041D000E9010E94D01E0AC06AE08091E9010E94B4
:1041E000461F04C01092EA0180E004C081E002C0D2
:1041F00080E0ABCFCF910895E1E8F0E08081886066
:1042000080838081816080838FB7F89493E090935E
:10421000890090ED909388008FBF0895EFE6F0E05D
:104220008081826080830895EFE6F0E080818D7F59
:1042300080830895EFE6F0E0908182E08927808313
:1042400008951F920F920FB60F9211242F933F9350
:104250004F935F936F937F938F939F93AF93BF938E
:10426000EF93FF938091EB019091EC010196909375
:10427000EC018093EB01811103C082E00E941608DB
:10428000E091EC01E695E695F0E0E05AFC4FE49110
:104290008091EB018E1303C080E00E941608FF910D
:1042A000EF91BF91AF919F918F917F916F915F91AE
:1042B0004F913F912F910F900FBE0F901F90189527
:1042C00004D06894B1118DC0089570D088F09F57C4
:1042D00090F0B92F9927B751A0F0D1F0660F771F52
:1042E000881F991F1AF0BA95C9F712C0B13081F032
:1042F00077D0B1E0089574C0672F782F8827B85F12
:1043000039F0B93FCCF3869577956795B395D9F792
:104310003EF490958095709561957F4F8F4F9F4F9C
:104320000895E89409C097FB3EF4909580957095A8
:1043300061957F4F8F4F9F4F9923A9F0F92F96E9F1
:10434000BB279395F695879577956795B795F11166
:10435000F8CFFAF4BB0F11F460FF1BC06F5F7F4F03
:104360008F4F9F4F16C0882311F096E911C0772315
:1043700021F09EE8872F762F05C0662371F096E81E
:10438000862F70E060E02AF09A95660F771F881FED
:10439000DAF7880F9695879597F9089557FD905805
:1043A000440F551F59F05F3F71F04795880F97FBF9
:1043B000991F61F09F3F79F08795089512161306B3
:1043C0001406551FF2CF4695F1DF08C016161706E2
:1043D0001806991FF1CF8695710561050894089517
:1043E000E894BB2766277727CB0197F908950BD070
:1043F00078C069D028F06ED018F0952309F05AC023
:104400005FC01124EECFCADFA0F3959FD1F3950FC3
:1044100050E0551F629FF001729FBB27F00DB11D48
:10442000639FAA27F00DB11DAA1F649F6627B00DD8
:10443000A11D661F829F2227B00DA11D621F739FC1
:10444000B00DA11D621F839FA00D611D221F749FCF
:104450003327A00D611D231F849F600D211D822F16
:10446000762F6A2F11249F5750408AF0E1F088235D
:104470004AF0EE0FFF1FBB1F661F771F881F91506A
:104480005040A9F79E3F510570F014C0AACF5F3F7E
:10449000ECF3983EDCF3869577956795B795F7959D
:1044A000E7959F5FC1F7FE2B880F911D9695879525
:1044B00097F9089597F99F6780E870E060E00895A4
:1044C0009FEF80EC089500240A941616170618062C
:1044D0000906089500240A94121613061406050608
:1044E0000895092E0394000C11F4882352F0BB0F99
:1044F00040F4BF2B11F460FF04C06F5F7F4F8F4FFC
:104500009F4F089597FB072E16F4009407D077FD70
:1045100009D00E949C2207FC05D03EF4909581951D
:104520009F4F0895709561957F4F0895EE0FFF1F7F
:104530000590F491E02D0994AA1BBB1B51E107C023
:10454000AA1FBB1FA617B70710F0A61BB70B881F23
:10455000991F5A95A9F780959095BC01CD010895B2
:10456000F999FECF92BD81BDF89A992780B508953B
:10457000A8E1B0E042E050E00C94D822262FF9994F
:10458000FECF92BD81BDF89A019700B4021639F0B2
:104590001FBA20BD0FB6F894FA9AF99A0FBE089583
:1045A0000196272F0E94BF220C94BE22DC01CB0172
:1045B000FC01F999FECF06C0F2BDE1BDF89A319633
:1045C00000B40D9241505040B8F70895F894FFCFD1
:1045D00002201808A60883084F081B080101C7011C
:1045E00028080A03140A3F4D36392103D4029E02DB
:1045F0006502F80111022A024302010203040506C2
:04460000070809009E
:00000001FF
